:1000000012C02CC02BC02AC029C028C027C026C0BF
:1000100025C024C023C022C021C020C01FC01EC0D4
:100020001DC01CC01BC011241FBECFE5D4E0DEBF25
:10003000CDBF10E0A0E6B0E0EAE5F1E002C0059037
:100040000D92A036B107D9F710E0A0E6B0E001C0EC
:100050001D92A036B107E1F723D07EC0D1CF97988B
:10006000969880EA8A95F1F79798969A8AE08A9509
:10007000F1F70895979896988AE08A95F1F79798FE
:10008000969A80EA8A95F1F70895979896988AE16A
:100090008A95F1F79798969A85E28A95F1F70895EF
:1000A000CF93DF938FEF81BBC0E0D0E082E0C23717
:1000B000D80719F4C1E0D0E02AC0219681E0C93305
:1000C000D80790F481E0C733D80728F5C330D105AD
:1000D00001F1C430D10520F4C130D10510F117C0B1
:1000E000C630D105F0F417C081E0CE33D80748F40C
:1000F00081E0CC33D80778F481E0C933D80739F4EC
:100100000DC0CE018F569240039758F404C0A7DF6C
:1001100006C0A5DF01C0AEDFADDFC8CFABDF9FDF1C
:10012000C5CFB3DF979A96988AE2982F9A95F1F700
:100130009798969A9AE4292F2A95F1F7979A969A82
:10014000282F2A95F1F79798969A9A95F1F7979A0A
:0A01500096988A95F1F7AACFFFCF29
:00000001FF
